:0A000000862B00000000000000281D
:10000A0083120313FB01FA01F901F801C301730D0D
:10001A00F80D7408F8027508031C750FF9027608C2
:10002A00031C760FFA027708031C770FFB02000104
:10003A00031C0130C302F30D0730FC00730DF80DE9
:10004A00F90DFA0DFB0DC30D7408731C3E28F80256
:10005A007508031C750FF9027608031C760FFA025D
:10006A007708031C770FFB020001031C0130C3024F
:10007A004F28F80775080318750FF907760803184B
:10008A00760FFA0777080318770FFB0700010318A2
:10009A000130C307F30DFC0B2328720DF80DF90D7F
:1000AA00FA0DFB0DC30D7408731C6D28F802750850
:1000BA00031C750FF9027608031C760FFA027708FB
:1000CA00031C770FFB020001031C0130C3027E28C8
:1000DA00F80775080318750FF90776080318760FDD
:1000EA00FA0777080318770FFB0700010318013096
:1000FA00C307F20D0730FC00720DF80DF90DFA0D69
:10010A00FB0DC30D7408721C9C28F8027508031CA9
:10011A00750FF9027608031C760FFA027708031C9A
:10012A00770FFB020001031C0130C302AD28F80758
:10013A0075080318750FF90776080318760FFA077A
:10014A0077080318770FFB07000103180130C3076C
:10015A00F20DFC0B8128710DF80DF90DFA0DFB0D4E
:10016A00C30D7408721CCB28F8027508031C750F9E
:10017A00F9027608031C760FFA027708031C770F38
:10018A00FB020001031C0130C302DC28F8077508D2
:10019A000318750FF90776080318760FFA07770818
:1001AA000318770FFB07000103180130C307F10D8D
:1001BA000730FC00710DF80DF90DFA0DFB0DC30D9A
:1001CA007408711CFA28F8027508031C750FF902E5
:1001DA007608031C760FFA027708031C770FFB02D6
:1001EA000001031C0130C3020B29F8077508031824
:1001FA00750FF90776080318760FFA0777080318B8
:10020A00770FFB07000103180130C307F10DFC0B40
:10021A00DF28700DF80DF90DFA0DFB0DC30D7408EA
:10022A00711C2929F8027508031C750FF902760852
:10023A00031C760FFA027708031C770FFB020001F2
:10024A00031C0130C3023A29F80775080318750F11
:10025A00F90776080318760FFA0777080318770F55
:10026A00FB07000103180130C307F00D0730FC003B
:10027A00700DF80DF90DFA0DFB0DC30D7408701C05
:10028A005829F8027508031C750FF9027608031C31
:10029A00760FFA027708031C770FFB020001031C92
:1002AA000130C3026929F80775080318750FF907A1
:1002BA0076080318760FFA0777080318770FFB07F3
:1002CA00000103180130C307F00DFC0B3D2970181B
:1002DA007C297408F80775080318750FF90776085A
:1002EA000318760FFA0777080318770FFB07080039
:1002FA007408F8027508031C750FF9027608031CC6
:10030A00760FFA027708031C770FFB02F30D07300A
:10031A00FC00730DF80DF90DFA0DFB0D7408731C32
:10032A00A429F8027508031C750FF9027608031C44
:10033A00760FFA027708031C770FFB02B129F80738
:10034A0075080318750FF90776080318760FFA0768
:10035A0077080318770FFB07F30DFC0B8E29720D34
:10036A00F80DF90DFA0DFB0D7408731CCA29F80271
:10037A007508031C750FF9027608031C760FFA023A
:10038A007708031C770FFB02D729F80775080318AB
:10039A00750FF90776080318760FFA077708031816
:1003AA00770FFB07F20D0730FC00720DF80DF90DFF
:1003BA00FA0DFB0D7408721CF029F8027508031C6B
:1003CA00750FF9027608031C760FFA027708031CE8
:1003DA00770FFB02FD29F80775080318750FF9074F
:1003EA0076080318760FFA0777080318770FFB07C2
:1003FA00F20DFC0BDA29710DF80DF90DFA0DFB0D52
:10040A007408721C162AF8027508031C750FF90283
:10041A007608031C760FFA027708031C770FFB0293
:10042A00232AF80775080318750FF90776080318C1
:10043A00760FFA0777080318770FFB07F10D0730D5
:10044A00FC00710DF80DF90DFA0DFB0D7408711C05
:10045A003C2AF8027508031C750FF9027608031C7A
:10046A00760FFA027708031C770FFB02492AF8076E
:10047A0075080318750FF90776080318760FFA0737
:10048A0077080318770FFB07F10DFC0B262A700D6E
:10049A00F80DF90DFA0DFB0D7408711C622AF802A9
:1004AA007508031C750FF9027608031C760FFA0209
:1004BA007708031C770FFB026F2AF80775080318E1
:1004CA00750FF90776080318760FFA0777080318E5
:1004DA00770FFB07F00D0730FC00700DF80DF90DD2
:1004EA00FA0DFB0D7408701C882AF8027508031CA3
:1004FA00750FF9027608031C760FFA027708031CB7
:10050A00770FFB02952AF80775080318750FF90784
:10051A0076080318760FFA0777080318770FFB0790
:10052A00F00DFC0B722A7018A82A7408F8077508CF
:10053A000318750FF90776080318760FFA07770874
:08054A000318770FFB070800FE
:1005520083124A08C4004B08F0000130F200700810
:100562000319B72AF20D7210FF3EB12A7208C600B3
:100572007209C5004C08F1000130F000710803193E
:10058200C62AF00D7010FF3EC02A7008BE00F009A6
:100592007008BD0080304A07840072088004700829
:1005A2008005BF0151080319D72ABF0984133F08E8
:1005B200003A0319DF2A3D088005E12A3E0880043B
:1005C200C727E830F4000330F500F601F70188266A
:1005D2007008D2007108D3007208D4007308D500E5
:1005E2004D08F0004E08F1004F08F2005008F300E9
:1005F200F00DF10DF20DF30D7010F00DF10DF20D85
:10060200F30D70100A30F400F501F601F7018826A7
:100612007008D6007108D7007208D8007308D90094
:100622007008F4007108F5007208F6007308F7000C
:100632005208F0005308F1005408F2005508F30084
:100642004B247008DA007108DB007108F400F50130
:10065200740875040319302B0230F00008005A08A0
:10066200C1005608F4005708F5005808F60059086A
:10067200F7005208F0005308F1005408F200550840
:10068200F3004B247808F0007908F1007A08F200B0
:100692007B08F3007008D2007108D3007208D400FE
:1006A2007308D5005608F5005708F6005808F700F9
:1006B2005908F800F80CF70CF60CF50CF813781B37
:1006C200F81780307806F400803073067402031D38
:1006D200742B72087702031D742B71087602031DB6
:1006E200742B700875020318772BC10A4108F100B8
:1006F200F10CF1137108C000073071020318842B4A
:0A0702000130F0000800F0010800CB
:10070C0021308312A0003030A1003130A2003230F1
:10071C00A3003330A4003430A5003530A6003630A9
:10072C00A7003730A8003830A9003930AA00303083
:10073C00AB003130AC003230AD003330AE00343071
:10074C00AF003530B0003630B100B2016A278512E7
:10075C000530CA00003005180130CB000030851878
:10076C000130CC008030CD002530CE00CF01D0013F
:10077C00D101A9227008B500CF27CA01CB01BF2631
:10078C00CF2785168519CB2B9327B7010C30B600D4
:10079C00B8018C30C7003030CA000030CB00BF2607
:1007AC00B301B401E52B2030B700062C4030B70064
:1007BC00062C6030B700062CB701062C062C003036
:1007CC003406031DEB2B003033060319D92B0030F4
:1007DC003406031DF32B013033060319DC2B0030D8
:1007EC003406031DFB2B023033060319DF2B0030BC
:1007FC003406031D032C033033060319E22BE42BC0
:10080C005630DC004F2630303307DC004F263D30AD
:10081C00DC004F264030B900E230BA000130BB009A
:10082C000030BC0085191B2CB2253908CA003A08C7
:10083C00CB003B08CC003C08CD002008CE00E524C2
:10084C002008CA002C272C30DC004F260330FB007C
:10085C00CB30FC004530FD00FD0B322CFC0B322C58
:10086C00FB0B322CB30A0319B40A80303406F000A7
:10087C0080307002031D442C04303302031CD82B2F
:0A088C00CF2720308506D62B4A2C1A
:1008960083120313FC01F71BFC0AFD01FB01FA019D
:1008A600F901F80173087204710470040319DF2C4E
:1008B60073087706C300C31BFD09F71F6D2CF409E7
:1008C600F509F609F709F40A0319F50A0319F60AF0
:1008D6000319F70AF31F7A2CF009F109F209F30953
:1008E600F00A0319F10A0319F20A0319F30A730845
:1008F6007704C300C31B9B2C7D21FC1BB82CFD1F5A
:10090600DF2CF009F109F209F309F00A0319F10ADB
:100916000319F20A0319F30AF809F909FA09FB0996
:10092600F80A0319F90A0319FA0A0319FB0ADF2C54
:10093600F71FB22CF31BAC2C7308FB007208FA00ED
:100946007108F9007008F800F301F201F101F001F5
:10095600822CF301F201F101F001F00A0034F309EF
:10096600F209F109F009FC177F2CF80A0319F90AB4
:100976000319FA0A0319FB0A74087802031D822C6C
:1009860075087902031D822C76087A02031D822CD3
:1009960077087B02031D822CFB01FA01F901F8019D
:1009A600F00A0319F10A0319F20A0319F30AF31FED
:1009B600822CC3014316FF34C3017C1CE32C87271A
:0409C600003E0800E7
:1009CA008312CF01D00100305002031DEE2C0A30F1
:1009DA004F020318F92C4F084E078400203080007C
:1009EA00CF0A0319D00AE82C4F084E078400800169
:1009FA000130CF02031CD0034F084E07D1000A3042
:100A0A00F400F501F601F7014A08F0004B08F1007D
:100A1A004C08F2004D08F30005207808F000790828
:100A2A00F1007A08F2007B08F30030307007F40016
:100A3A0051088400740880000A30F400F501F601B8
:100A4A00F7014A08F0004B08F1004C08F2004D0883
:100A5A00F30005207008CA007108CB007208CC00A8
:100A6A007308CD000030F4007306031D462D740888
:100A7A007206031D462D74087106031D462D700863
:100A8A00003A031D492D4E2D0130CF02031CD0031D
:040A9A00012D080022
:100A9E0001308312DD000030DE008030DF00E00127
:100AAE005F08600403197F2DDD27DD27DD27DD2795
:100ABE00AA270512DD27DD275F085C05F000003050
:100ACE006005F1007008710403196F2D0515712D65
:100ADE00B4270511DD27DD2705164210051A7B2DDB
:100AEE00421C7A2D7B2D752DE00CDF0CE013572D5B
:100AFE00DD01DE01DD27DD27AA270512DD27DD2733
:100B0E000515DD27DD27DD27DD2705164210051A21
:100B1E00942D421C932D942D8E2DDD01DE01DD27AB
:100B2E00DD27051D9B2D5D14DD27DD27DD27DD2748
:100B3E00DD27DD27DD27DD27DD27DD27DD27DD2787
:100B4E00DD27DD27DD27DD27AA270512B4270511AE
:060B5E005D08F000080034
:100B64008312CA01CB01CC01CD014A30CE00370833
:100B7400803EC7003608C7073808C70779274230C0
:100B8400FD00FD0BC32D0000D030DC004F254230AA
:100B9400FD00FD0BCB2D00004708DC004F2514277A
:100BA4007927D130DC004F2503304E0784008001C3
:100BB40002304E07CF000130DC000030DD000B2690
:100BC4000330F0054F088400700880004E0ACF00FF
:100BD4000130DC000030DD000B264F088400700873
:100BE40080004E08CF000130DC000030DD000B2611
:100BF4004F08840070088000DC01DD010B261427F7
:100C04004A08B9004B08BA004C08BB004D08BC00A8
:020C14000800D6
:100C160080308312DE000030DF00E001E1015E0873
:100C26005F040319312EDD27DD270515DD27DD27B6
:100C360005164210051A232E421C222E232E1D2E87
:100C4600051D292E5E08E0045F08E104DD27DD2787
:100C5600AA270512DF0CDE0CDF13122E0515DD2781
:100C6600DD275C085D0403193A2EB4270511DD273C
:100C7600DD2705164210051A442E421C432E442E2B
:100C86003E2EDD27DD27AA270512DD27DD27B4271F
:080C960005116008F0000800E0
:100C9E0001308312DD003F08DC06440884003F0863
:100CAE00003A03195D2E3E0880045F2E3D08800534
:100CBE004108E2005827DC095D0803197B2E5D0808
:100CCE005C05F000031D6E2E3E088004702E3D085C
:100CDE008005DD0D5D1002304102E2005827000054
:100CEE00000000000000632E3F08003A0319822E18
:100CFE003D088005842E3E0880044108E2005827F6
:020D0E000800DB
:100D1000831203132230FC00F801F901FA01FB01F0
:100D2000FC030319BE2E0310FB0CFA0CF90CF80C93
:100D3000F30CF20CF10CF00C031C902EFC030319C5
:100D4000B02E7408F80775080318750FF9077608B0
:100D50000318760FFA0777080318770FFB07942E0E
:100D60007408F80775080318750FF9077608031853
:0E0D7000760FFA0777080318770FFB070800C5
:100D7E0083124A08CC004B08CD004C08DC00BE277D
:100D8E0070088312CE00CF0100304F06031DD12E06
:100D9E0000304E06031DD42EF52E2030DC0003301D
:100DAE00DD00DE01DF01F6264E08DC004F26CC0A00
:100DBE000319CD0A8030F00080304D067002031DFD
:100DCE00EA2E4C08FF3C0318ED2EF52E00304F0690
:0E0DDE00031DF32E00304E06031DC42E080028
:100DEC0080308312F00080305F067002031D082FE4
:100DFC005E08003C031D082F5D08003C031D082FF6
:100E0C005C08003C0318132F0130DC02031CDD02CC
:0C0E1C00031CDE02031CDF02F62E08009F
:100E2800B4270511DD27DD2705164210051A202FE6
:100E3800421C1F2F202F1A2FDD27DD27DD27DD2756
:100E4800DD27DD27DD27DD270515DD27DD27080060
:100E580083124A08DC0043277008CC00CB014B08FA
:100E68004A0784000008DC004F26CB0A80304B0676
:0E0E7800F00080304C067002031C332F08007F
:100E860083125C08F2007208F000F20A700884000F
:100E9600000803194F2F462F5C087202F00001303C
:0A0EA600F002F101031CF103080043
:100EB0008312E203E2036208003C0318642FE2039A
:100EC0000000000000005B2F000000000000000098
:040ED0000000080016
:100ED400753083168F0009308500343095009601F3
:0E0EE4009F0183121F10FF3099008B01080040
:100EF20083120515DD27DD270516DD27DD27B4273B
:0C0F02000511DD27DD27AA2705120800D5
:100F0E00FB09FA09F909F809F80A0319F90A03198C
:080F1E00FA0A0319FB0A08009E
:100F26008312051605154210051A9D2F421C9C2F8B
:060F36009D2F972F08001B
:100F3C00D7278A110A128000840AC80A0319C90A21
:080F4C00F003031D9E2F0800B5
:100F540005308400000800088312F0007012700845
:040F64008000080001
:100F680005308400000800088312F0007011700832
:040F780080000800ED
:100F7C0083125C0883169B009C131C141A08F00047
:020F8C0008005B
:100F8E0040308312F0001F30F100F201F30108002F
:100F9E000A308312DC004F260D30DC004F2608008D
:0C0FAE00831249088A00480882000800ED
:060FBA0000000000080029
:02400E00C400EC
:104200002000560065007200730069006F006E00A8
:1042100020003100330020006A0061006E0076004B
:1042200020003200300031003100200050006100D9
:1042300075006C0046006A0075006A006F0020007F
:104240003100320046003600380033005F00330092
:1042500065006D002E0043002000200020000000BB
:104260004100440043002000310038006200690032
:104270007400730020004D004300500033003400F0
:104280003200340020002000310037006200690055
:10429000740073000D000A004D0061007800690091
:1042A0003D00310033003100300037003100200084
:1042B000500074007300200070006F0075007200E1
:1042C000200032002C00300034003800200056005E
:1042D0006F006C00740073000D000A000000000005
:1042E000FF00FF00FF00FF00FF00FF00FF00FF00D6
:1042F000FF00FF00FF00FF00FF00FF00FF00FF00C6
:104300007000610075006C0066006A0075006A004C
:104310006F000000FF00FF00FF00FF00FF00FF0034
:1043200052005300320033003200200039003600C2
:10433000300030000000FF00FF00FF00FF00FF0022
:104340007200FF00FF00FF00FF00FF00FF00FF0002
:10435000FF00FF00FF00FF00FF00FF00FF00FF0065
:10436000FF00FF00FF00FF00FF00FF00FF00FF0055
:10437000FF00FF00FF00FF00FF00FF00FF00FF0045
:10438000FF00FF00FF00FF00FF00FF00FF00FF0035
:10439000FF00FF00FF00FF00FF00FF00FF00FF0025
:1043A000FF00FF00FF00FF00FF00FF00FF00FF0015
:1043B000FF00FF00FF00FF00FF00FF00FF00FF0005
:1043C000FF00FF00FF00FF00FF00FF00FF00FF00F5
:1043D000FF00FF00FF00FF00FF00FF00FF00FF00E5
:1043E000FF00FF00FF00FF00FF00FF00FF00FF00D5
:1043F000FF00FF00FF00FF00FF00FF00FF00FF00C5
:00000001FF
